 getlocal003

 Timestamp is b57fba1e (reproducible build file hash)

 Preferred load address is 0000000180000000

 Start         Length     Name                   Class
 0001:00000000 00003500H .text$mn                CODE
 0001:00003500 00000036H .text$mn$00             CODE
 0001:00003536 00000092H .text$x                 CODE
 0002:00000000 00000198H .idata$5                DATA
 0002:00000198 00000038H .00cfg                  DATA
 0002:000001d0 00000008H .CRT$XCA                DATA
 0002:000001d8 00000008H .CRT$XCZ                DATA
 0002:000001e0 00000008H .CRT$XIA                DATA
 0002:000001e8 00000008H .CRT$XIC                DATA
 0002:000001f0 00000008H .CRT$XIZ                DATA
 0002:000001f8 00000008H .CRT$XLA                DATA
 0002:00000200 00000008H .CRT$XLZ                DATA
 0002:00000208 00000008H .CRT$XPA                DATA
 0002:00000210 00000008H .CRT$XPZ                DATA
 0002:00000218 00000008H .CRT$XTA                DATA
 0002:00000220 00000010H .CRT$XTZ                DATA
 0002:00000228 00000000H .gehcont$y              DATA
 0002:00000228 00000000H .gfids$y                DATA
 0002:00000230 000024d0H .rdata                  DATA
 0002:00002700 00000000H .rdata$CastGuardVftablesA DATA
 0002:00002700 00000000H .rdata$CastGuardVftablesC DATA
 0002:00002700 00000028H .rdata$T                DATA
 0002:00002728 000000a4H .rdata$voltmd           DATA
 0002:000027cc 0000031cH .rdata$zzzdbg           DATA
 0002:00002ae8 00000008H .rtc$IAA                DATA
 0002:00002af0 00000008H .rtc$IZZ                DATA
 0002:00002af8 00000008H .rtc$TAA                DATA
 0002:00002b00 00000008H .rtc$TZZ                DATA
 0002:00002b08 00000004H .tls                    DATA
 0002:00002b0c 00000004H .tls$                   DATA
 0002:00002b10 00000008H .tls$ZZZ                DATA
 0002:00002b18 00000328H .xdata                  DATA
 0002:00002e40 00000470H .edata                  DATA
 0002:000032b0 00000064H .idata$2                DATA
 0002:00003314 00000014H .idata$3                DATA
 0002:00003328 00000198H .idata$4                DATA
 0002:000034c0 0000041eH .idata$6                DATA
 0003:00000000 00000080H .data                   DATA
 0003:00000080 0001b398H .bss                    DATA
 0004:00000000 000003b4H .pdata                  DATA

  Address         Publics by Value              Rva+Base               Lib:Object

 0000:00000000       __AbsoluteZero             0000000000000000     <absolute>
 0000:00000000       ___safe_se_handler_count   0000000000000000     <absolute>
 0000:00000000       ___safe_se_handler_table   0000000000000000     <absolute>
 0000:00000000       __arm64x_extra_rfe_table   0000000000000000     <absolute>
 0000:00000000       __arm64x_extra_rfe_table_size 0000000000000000     <absolute>
 0000:00000000       __arm64x_native_entrypoint 0000000000000000     <absolute>
 0000:00000000       __arm64x_redirection_metadata 0000000000000000     <absolute>
 0000:00000000       __arm64x_redirection_metadata_count 0000000000000000     <absolute>
 0000:00000000       __dynamic_value_reloc_table 0000000000000000     <absolute>
 0000:00000000       __enclave_config           0000000000000000     <absolute>
 0000:00000000       __guard_check_icall_a64n_fptr 0000000000000000     <absolute>
 0000:00000000       __guard_eh_cont_count      0000000000000000     <absolute>
 0000:00000000       __guard_eh_cont_table      0000000000000000     <absolute>
 0000:00000000       __guard_fids_count         0000000000000000     <absolute>
 0000:00000000       __guard_fids_table         0000000000000000     <absolute>
 0000:00000000       __guard_iat_count          0000000000000000     <absolute>
 0000:00000000       __guard_iat_table          0000000000000000     <absolute>
 0000:00000000       __guard_longjmp_count      0000000000000000     <absolute>
 0000:00000000       __guard_longjmp_table      0000000000000000     <absolute>
 0000:00000000       __hybrid_auxiliary_iat     0000000000000000     <absolute>
 0000:00000000       __hybrid_auxiliary_iat_copy 0000000000000000     <absolute>
 0000:00000000       __hybrid_code_map          0000000000000000     <absolute>
 0000:00000000       __hybrid_code_map_count    0000000000000000     <absolute>
 0000:00000000       __x64_code_ranges_to_entry_points 0000000000000000     <absolute>
 0000:00000000       __x64_code_ranges_to_entry_points_count 0000000000000000     <absolute>
 0000:00000100       __guard_flags              0000000000000100     <absolute>
 0000:00000000       __ImageBase                0000000180000000     <linker-defined>
 0001:00000000       ?NewObject@JNIEnv_@@QEAAPEAV_jobject@@PEAV_jclass@@PEAU_jmethodID@@ZZ 0000000180001000 f i libgetlocal003.obj
 0001:00000028       ?SetEventNotificationMode@_jvmtiEnv@@QEAA?AW4jvmtiError@@W4jvmtiEventMode@@W4jvmtiEvent@@PEAV_jobject@@ZZ 0000000180001028 f i libgetlocal003.obj
 0001:00000034       ?TranslateError@@YAPEBDW4jvmtiError@@@Z 0000000180001034 f   libgetlocal003.obj
 0001:000002ec       ?nsk_jni_check_exception@@YAHPEAUJNIEnv_@@QEBDH@Z 00000001800012ec f   libgetlocal003.obj
 0001:00000430       ?nsk_jni_lverify@@YAHHPEAUJNIEnv_@@HQEBDH1ZZ 0000000180001430 f   libgetlocal003.obj
 0001:000004d0       Agent_Initialize           00000001800014d0 f   libgetlocal003.obj
 0001:00000658       Agent_OnAttach             0000000180001658 f   libgetlocal003.obj
 0001:00000658       Agent_OnLoad               0000000180001658 f   libgetlocal003.obj
 0001:00000660       Java_nsk_jvmti_unit_FollowReferences_FollowRefObjects_addRefToVerify 0000000180001660 f   libgetlocal003.obj
 0001:00000838       Java_nsk_jvmti_unit_FollowReferences_FollowRefObjects_getTag 0000000180001838 f   libgetlocal003.obj
 0001:000008f8       Java_nsk_jvmti_unit_FollowReferences_FollowRefObjects_resetRefsToVerify 00000001800018f8 f   libgetlocal003.obj
 0001:00000900       Java_nsk_jvmti_unit_FollowReferences_FollowRefObjects_resetTags 0000000180001900 f   libgetlocal003.obj
 0001:00000944       Java_nsk_jvmti_unit_FollowReferences_FollowRefObjects_setTag 0000000180001944 f   libgetlocal003.obj
 0001:00000b9c       Java_nsk_jvmti_unit_GetLocalVariable_getlocal003_checkLoc 0000000180001b9c f   libgetlocal003.obj
 0001:00000e58       Java_nsk_jvmti_unit_GetLocalVariable_getlocal003_getMeth 0000000180001e58 f   libgetlocal003.obj
 0001:00001030       Java_nsk_jvmti_unit_GetLocalVariable_getlocal003_getRes 0000000180002030 f   libgetlocal003.obj
 0001:00001038       Java_nsk_jvmti_unit_GetLocalVariable_getlocal003_instMeth 0000000180002038 f   libgetlocal003.obj
 0001:00001188       Java_nsk_share_jvmti_ArgumentHandler_getAgentOptionsString 0000000180002188 f   libgetlocal003.obj
 0001:00001238       Java_nsk_share_jvmti_DebugeeClass_checkStatus 0000000180002238 f   libgetlocal003.obj
 0001:000012c0       Java_nsk_share_jvmti_DebugeeClass_resetAgentData 00000001800022c0 f   libgetlocal003.obj
 0001:00001320       Java_nsk_share_jvmti_RedefineAgent_agentStatus 0000000180002320 f   libgetlocal003.obj
 0001:0000132c       Java_nsk_share_jvmti_RedefineAgent_isRedefined 000000018000232c f   libgetlocal003.obj
 0001:00001338       Java_nsk_share_jvmti_RedefineAgent_redefineAttempted 0000000180002338 f   libgetlocal003.obj
 0001:00001344       MA_checkStatus             0000000180002344 f   libgetlocal003.obj
 0001:000014dc       __local_stdio_printf_options 00000001800024dc f i libgetlocal003.obj
 0001:000016bc       exitOnError                00000001800026bc f   libgetlocal003.obj
 0001:00001770       fprintf                    0000000180002770 f i libgetlocal003.obj
 0001:000017b4       nsk_jvmti_lverify          00000001800027b4 f   libgetlocal003.obj
 0001:000018a4       nsk_jvmti_resetAgentData   00000001800028a4 f   libgetlocal003.obj
 0001:00001924       nsk_jvmti_setFailStatus    0000000180002924 f   libgetlocal003.obj
 0001:00001960       nsk_lcomplain              0000000180002960 f   libgetlocal003.obj
 0001:00001980       nsk_ldisplay               0000000180002980 f   libgetlocal003.obj
 0001:000019a0       nsk_ltrace                 00000001800029a0 f   libgetlocal003.obj
 0001:000019c0       nsk_lvcomplain             00000001800029c0 f   libgetlocal003.obj
 0001:00001b78       nsk_lvdisplay              0000000180002b78 f   libgetlocal003.obj
 0001:00001bc4       nsk_lverify                0000000180002bc4 f   libgetlocal003.obj
 0001:00001c20       nsk_lvtrace                0000000180002c20 f   libgetlocal003.obj
 0001:00001c80       nsk_printf                 0000000180002c80 f   libgetlocal003.obj
 0001:00001ca8       nsk_vprintf                0000000180002ca8 f   libgetlocal003.obj
 0001:00001d5c       print_LocalVariableEntry   0000000180002d5c f   libgetlocal003.obj
 0001:00001db0       printf                     0000000180002db0 f i libgetlocal003.obj
 0001:000025d4       __raise_securityfailure    00000001800035d4 f   MSVCRT:gs_report.obj
 0001:00002608       __report_gsfailure         0000000180003608 f   MSVCRT:gs_report.obj
 0001:00002848       __GSHandlerCheck           0000000180003848 f   MSVCRT:gshandler.obj
 0001:00002868       __GSHandlerCheckCommon     0000000180003868 f   MSVCRT:gshandler.obj
 0001:000028e0       __security_check_cookie    00000001800038e0 f   MSVCRT:amdsecgs.obj
 0001:00002c20       _DllMainCRTStartup         0000000180003c20 f   MSVCRT:dll_dllmain.obj
 0001:00002c60       __scrt_acquire_startup_lock 0000000180003c60 f   MSVCRT:utility.obj
 0001:00002c9c       __scrt_dllmain_after_initialize_c 0000000180003c9c f   MSVCRT:utility.obj
 0001:00002cd0       __scrt_dllmain_before_initialize_c 0000000180003cd0 f   MSVCRT:utility.obj
 0001:00002ce8       __scrt_dllmain_crt_thread_attach 0000000180003ce8 f   MSVCRT:utility.obj
 0001:00002d10       __scrt_dllmain_crt_thread_detach 0000000180003d10 f   MSVCRT:utility.obj
 0001:00002d28       __scrt_dllmain_exception_filter 0000000180003d28 f   MSVCRT:utility.obj
 0001:00002d88       __scrt_dllmain_uninitialize_c 0000000180003d88 f   MSVCRT:utility.obj
 0001:00002db8       __scrt_dllmain_uninitialize_critical 0000000180003db8 f   MSVCRT:utility.obj
 0001:00002dcc       __scrt_initialize_crt      0000000180003dcc f   MSVCRT:utility.obj
 0001:00002e18       __scrt_initialize_onexit_tables 0000000180003e18 f   MSVCRT:utility.obj
 0001:00002ea4       __scrt_is_nonwritable_in_current_image 0000000180003ea4 f   MSVCRT:utility.obj
 0001:00002f3c       __scrt_release_startup_lock 0000000180003f3c f   MSVCRT:utility.obj
 0001:00002f60       __scrt_uninitialize_crt    0000000180003f60 f   MSVCRT:utility.obj
 0001:00002f8c       _onexit                    0000000180003f8c f   MSVCRT:utility.obj
 0001:00002fc8       atexit                     0000000180003fc8 f   MSVCRT:utility.obj
 0001:00002fe0       __crt_debugger_hook        0000000180003fe0 f   MSVCRT:utility_desktop.obj
 0001:00002fe8       __scrt_fastfail            0000000180003fe8 f   MSVCRT:utility_desktop.obj
 0001:00003134       _guard_check_icall_nop     0000000180004134 f i MSVCRT:guard_support.obj
 0001:00003138       __security_init_cookie     0000000180004138 f   MSVCRT:gs_support.obj
 0001:000031e4       DllMain                    00000001800041e4 f   MSVCRT:dll_dllmain_stub.obj
 0001:00003208       ?__scrt_initialize_type_info@@YAXXZ 0000000180004208 f   MSVCRT:tncleanup.obj
 0001:00003218       ?__scrt_uninitialize_type_info@@YAXXZ 0000000180004218 f   MSVCRT:tncleanup.obj
 0001:00003224       __local_stdio_scanf_options 0000000180004224 f i MSVCRT:default_local_stdio_options.obj
 0001:0000322c       __scrt_initialize_default_local_stdio_options 000000018000422c f   MSVCRT:default_local_stdio_options.obj
 0001:00003248       __scrt_get_dyn_tls_init_callback 0000000180004248 f   MSVCRT:dyn_tls_init.obj
 0001:00003250       _RTC_Initialize            0000000180004250 f   MSVCRT:initsect.obj
 0001:0000328c       _RTC_Terminate             000000018000428c f   MSVCRT:initsect.obj
 0001:000032c8       __isa_available_init       00000001800042c8 f   MSVCRT:cpu_disp.obj
 0001:00003474       _get_startup_argv_mode     0000000180004474 f   MSVCRT:argv_mode.obj
 0001:0000347c       __scrt_is_ucrt_dll_in_use  000000018000447c f   MSVCRT:ucrt_detection.obj
 0001:00003490       memcpy                     0000000180004490 f   vcruntime:VCRUNTIME140.dll
 0001:00003496       memset                     0000000180004496 f   vcruntime:VCRUNTIME140.dll
 0001:0000349c       strchr                     000000018000449c f   vcruntime:VCRUNTIME140.dll
 0001:000034a2       __C_specific_handler       00000001800044a2 f   vcruntime:VCRUNTIME140.dll
 0001:000034a8       __std_type_info_destroy_list 00000001800044a8 f   vcruntime:VCRUNTIME140.dll
 0001:000034ae       strcmp                     00000001800044ae f   ucrt:api-ms-win-crt-string-l1-1-0.dll
 0001:000034b4       strlen                     00000001800044b4 f   ucrt:api-ms-win-crt-string-l1-1-0.dll
 0001:000034ba       _initterm                  00000001800044ba f   ucrt:api-ms-win-crt-runtime-l1-1-0.dll
 0001:000034c0       _initterm_e                00000001800044c0 f   ucrt:api-ms-win-crt-runtime-l1-1-0.dll
 0001:000034c6       _seh_filter_dll            00000001800044c6 f   ucrt:api-ms-win-crt-runtime-l1-1-0.dll
 0001:000034cc       _configure_narrow_argv     00000001800044cc f   ucrt:api-ms-win-crt-runtime-l1-1-0.dll
 0001:000034d2       _initialize_narrow_environment 00000001800044d2 f   ucrt:api-ms-win-crt-runtime-l1-1-0.dll
 0001:000034d8       _initialize_onexit_table   00000001800044d8 f   ucrt:api-ms-win-crt-runtime-l1-1-0.dll
 0001:000034de       _register_onexit_function  00000001800044de f   ucrt:api-ms-win-crt-runtime-l1-1-0.dll
 0001:000034e4       _execute_onexit_table      00000001800044e4 f   ucrt:api-ms-win-crt-runtime-l1-1-0.dll
 0001:000034ea       _crt_atexit                00000001800044ea f   ucrt:api-ms-win-crt-runtime-l1-1-0.dll
 0001:000034f0       _cexit                     00000001800044f0 f   ucrt:api-ms-win-crt-runtime-l1-1-0.dll
 0001:000034f8       __acrt_initialize          00000001800044f8 f   MSVCRT:ucrt_stubs.obj
 0001:000034f8       __acrt_thread_attach       00000001800044f8 f   MSVCRT:ucrt_stubs.obj
 0001:000034f8       __acrt_thread_detach       00000001800044f8 f   MSVCRT:ucrt_stubs.obj
 0001:000034f8       __acrt_uninitialize        00000001800044f8 f   MSVCRT:ucrt_stubs.obj
 0001:000034f8       __acrt_uninitialize_critical 00000001800044f8 f   MSVCRT:ucrt_stubs.obj
 0001:000034f8       __scrt_stub_for_acrt_initialize 00000001800044f8 f   MSVCRT:ucrt_stubs.obj
 0001:000034f8       __scrt_stub_for_acrt_thread_attach 00000001800044f8 f   MSVCRT:ucrt_stubs.obj
 0001:000034f8       __scrt_stub_for_acrt_thread_detach 00000001800044f8 f   MSVCRT:ucrt_stubs.obj
 0001:000034f8       __scrt_stub_for_acrt_uninitialize 00000001800044f8 f   MSVCRT:ucrt_stubs.obj
 0001:000034f8       __scrt_stub_for_acrt_uninitialize_critical 00000001800044f8 f   MSVCRT:ucrt_stubs.obj
 0001:000034f8       __vcrt_initialize          00000001800044f8 f   MSVCRT:ucrt_stubs.obj
 0001:000034f8       __vcrt_thread_attach       00000001800044f8 f   MSVCRT:ucrt_stubs.obj
 0001:000034f8       __vcrt_thread_detach       00000001800044f8 f   MSVCRT:ucrt_stubs.obj
 0001:000034f8       __vcrt_uninitialize        00000001800044f8 f   MSVCRT:ucrt_stubs.obj
 0001:000034f8       __vcrt_uninitialize_critical 00000001800044f8 f   MSVCRT:ucrt_stubs.obj
 0001:000034fc       __scrt_stub_for_is_c_termination_complete 00000001800044fc f   MSVCRT:ucrt_stubs.obj
 0001:000034fc       _is_c_termination_complete 00000001800044fc f   MSVCRT:ucrt_stubs.obj
 0001:00003510       _guard_dispatch_icall_nop  0000000180004510 f   MSVCRT:guard_dispatch.obj
 0001:00003530       _guard_xfg_dispatch_icall_nop 0000000180004530 f   MSVCRT:guard_xfg_dispatch.obj
 0002:00000000       __imp_RtlCaptureContext    0000000180005000     kernel32:KERNEL32.dll
 0002:00000008       __imp_RtlLookupFunctionEntry 0000000180005008     kernel32:KERNEL32.dll
 0002:00000010       __imp_RtlVirtualUnwind     0000000180005010     kernel32:KERNEL32.dll
 0002:00000018       __imp_UnhandledExceptionFilter 0000000180005018     kernel32:KERNEL32.dll
 0002:00000020       __imp_SetUnhandledExceptionFilter 0000000180005020     kernel32:KERNEL32.dll
 0002:00000028       __imp_GetCurrentProcess    0000000180005028     kernel32:KERNEL32.dll
 0002:00000030       __imp_TerminateProcess     0000000180005030     kernel32:KERNEL32.dll
 0002:00000038       __imp_IsProcessorFeaturePresent 0000000180005038     kernel32:KERNEL32.dll
 0002:00000040       __imp_CloseHandle          0000000180005040     kernel32:KERNEL32.dll
 0002:00000048       __imp_InitializeCriticalSectionAndSpinCount 0000000180005048     kernel32:KERNEL32.dll
 0002:00000050       __imp_DeleteCriticalSection 0000000180005050     kernel32:KERNEL32.dll
 0002:00000058       __imp_CreateEventW         0000000180005058     kernel32:KERNEL32.dll
 0002:00000060       __imp_GetModuleHandleW     0000000180005060     kernel32:KERNEL32.dll
 0002:00000068       __imp_GetProcAddress       0000000180005068     kernel32:KERNEL32.dll
 0002:00000070       __imp_IsDebuggerPresent    0000000180005070     kernel32:KERNEL32.dll
 0002:00000078       __imp_QueryPerformanceCounter 0000000180005078     kernel32:KERNEL32.dll
 0002:00000080       __imp_GetCurrentProcessId  0000000180005080     kernel32:KERNEL32.dll
 0002:00000088       __imp_GetCurrentThreadId   0000000180005088     kernel32:KERNEL32.dll
 0002:00000090       __imp_GetSystemTimeAsFileTime 0000000180005090     kernel32:KERNEL32.dll
 0002:00000098       __imp_DisableThreadLibraryCalls 0000000180005098     kernel32:KERNEL32.dll
 0002:000000a0       __imp_InitializeSListHead  00000001800050a0     kernel32:KERNEL32.dll
 0002:000000a8       \177KERNEL32_NULL_THUNK_DATA 00000001800050a8     kernel32:KERNEL32.dll
 0002:000000b0       __imp_memcpy               00000001800050b0     vcruntime:VCRUNTIME140.dll
 0002:000000b8       __imp_memset               00000001800050b8     vcruntime:VCRUNTIME140.dll
 0002:000000c0       __imp_strchr               00000001800050c0     vcruntime:VCRUNTIME140.dll
 0002:000000c8       __imp___C_specific_handler 00000001800050c8     vcruntime:VCRUNTIME140.dll
 0002:000000d0       __imp___std_type_info_destroy_list 00000001800050d0     vcruntime:VCRUNTIME140.dll
 0002:000000d8       \177VCRUNTIME140_NULL_THUNK_DATA 00000001800050d8     vcruntime:VCRUNTIME140.dll
 0002:000000e0       __imp__errno               00000001800050e0     ucrt:api-ms-win-crt-runtime-l1-1-0.dll
 0002:000000e8       __imp_exit                 00000001800050e8     ucrt:api-ms-win-crt-runtime-l1-1-0.dll
 0002:000000f0       __imp__cexit               00000001800050f0     ucrt:api-ms-win-crt-runtime-l1-1-0.dll
 0002:000000f8       __imp__crt_atexit          00000001800050f8     ucrt:api-ms-win-crt-runtime-l1-1-0.dll
 0002:00000100       __imp__execute_onexit_table 0000000180005100     ucrt:api-ms-win-crt-runtime-l1-1-0.dll
 0002:00000108       __imp__register_onexit_function 0000000180005108     ucrt:api-ms-win-crt-runtime-l1-1-0.dll
 0002:00000110       __imp__initialize_onexit_table 0000000180005110     ucrt:api-ms-win-crt-runtime-l1-1-0.dll
 0002:00000118       __imp__initialize_narrow_environment 0000000180005118     ucrt:api-ms-win-crt-runtime-l1-1-0.dll
 0002:00000120       __imp__configure_narrow_argv 0000000180005120     ucrt:api-ms-win-crt-runtime-l1-1-0.dll
 0002:00000128       __imp__seh_filter_dll      0000000180005128     ucrt:api-ms-win-crt-runtime-l1-1-0.dll
 0002:00000130       __imp__initterm_e          0000000180005130     ucrt:api-ms-win-crt-runtime-l1-1-0.dll
 0002:00000138       __imp__initterm            0000000180005138     ucrt:api-ms-win-crt-runtime-l1-1-0.dll
 0002:00000140       \177api-ms-win-crt-runtime-l1-1-0_NULL_THUNK_DATA 0000000180005140     ucrt:api-ms-win-crt-runtime-l1-1-0.dll
 0002:00000148       __imp___acrt_iob_func      0000000180005148     ucrt:api-ms-win-crt-stdio-l1-1-0.dll
 0002:00000150       __imp_fflush               0000000180005150     ucrt:api-ms-win-crt-stdio-l1-1-0.dll
 0002:00000158       __imp___stdio_common_vsprintf 0000000180005158     ucrt:api-ms-win-crt-stdio-l1-1-0.dll
 0002:00000160       __imp___stdio_common_vfprintf 0000000180005160     ucrt:api-ms-win-crt-stdio-l1-1-0.dll
 0002:00000168       \177api-ms-win-crt-stdio-l1-1-0_NULL_THUNK_DATA 0000000180005168     ucrt:api-ms-win-crt-stdio-l1-1-0.dll
 0002:00000170       __imp_strcmp               0000000180005170     ucrt:api-ms-win-crt-string-l1-1-0.dll
 0002:00000178       __imp__strdup              0000000180005178     ucrt:api-ms-win-crt-string-l1-1-0.dll
 0002:00000178       __imp_strdup               0000000180005178     ucrt:api-ms-win-crt-string-l1-1-0.dll
 0002:00000180       __imp_strlen               0000000180005180     ucrt:api-ms-win-crt-string-l1-1-0.dll
 0002:00000188       __imp_strncpy              0000000180005188     ucrt:api-ms-win-crt-string-l1-1-0.dll
 0002:00000190       \177api-ms-win-crt-string-l1-1-0_NULL_THUNK_DATA 0000000180005190     ucrt:api-ms-win-crt-string-l1-1-0.dll
 0002:00000198       __guard_check_icall_fptr   0000000180005198     MSVCRT:guard_support.obj
 0002:000001a0       __guard_xfg_check_icall_fptr 00000001800051a0     MSVCRT:guard_support.obj
 0002:000001a8       __guard_dispatch_icall_fptr 00000001800051a8     MSVCRT:guard_support.obj
 0002:000001b0       __guard_xfg_dispatch_icall_fptr 00000001800051b0     MSVCRT:guard_support.obj
 0002:000001b8       __guard_xfg_table_dispatch_icall_fptr 00000001800051b8     MSVCRT:guard_support.obj
 0002:000001c0       __castguard_check_failure_os_handled_fptr 00000001800051c0     MSVCRT:guard_support.obj
 0002:000001c8       __guard_memcpy_fptr        00000001800051c8     vcruntime:softmemtag.obj
 0002:000001d0       __xc_a                     00000001800051d0     MSVCRT:initializers.obj
 0002:000001d8       __xc_z                     00000001800051d8     MSVCRT:initializers.obj
 0002:000001e0       __xi_a                     00000001800051e0     MSVCRT:initializers.obj
 0002:000001f0       __xi_z                     00000001800051f0     MSVCRT:initializers.obj
 0002:000001f8       __xl_a                     00000001800051f8     MSVCRT:tlssup.obj
 0002:00000200       __xl_z                     0000000180005200     MSVCRT:tlssup.obj
 0002:00000208       __xp_a                     0000000180005208     MSVCRT:initializers.obj
 0002:00000210       __xp_z                     0000000180005210     MSVCRT:initializers.obj
 0002:00000218       __xt_a                     0000000180005218     MSVCRT:initializers.obj
 0002:00000220       __xt_z                     0000000180005220     MSVCRT:initializers.obj
 0002:00000230       g_refKindStr               0000000180005230     libgetlocal003.obj
 0002:000003e0       ??_C@_09BPLDFGCI@unknown_0@ 00000001800053e0     libgetlocal003.obj
 0002:000003f0       ??_C@_0BL@FPNMECJD@JVMTI_HEAP_REFERENCE_CLASS@ 00000001800053f0     libgetlocal003.obj
 0002:00000410       ??_C@_0BL@FKGKKLNM@JVMTI_HEAP_REFERENCE_FIELD@ 0000000180005410     libgetlocal003.obj
 0002:00000430       ??_C@_0CD@CAEHCFJF@JVMTI_HEAP_REFERENCE_ARRAY_ELEM@ 0000000180005430     libgetlocal003.obj
 0002:00000458       ??_C@_0CC@DNEBMCNK@JVMTI_HEAP_REFERENCE_CLASS_LOAD@ 0000000180005458     libgetlocal003.obj
 0002:00000480       ??_C@_0BN@CJMIPEBB@JVMTI_HEAP_REFERENCE_SIGNERS@ 0000000180005480     libgetlocal003.obj
 0002:000004a0       ??_C@_0CH@HBOIDPEB@JVMTI_HEAP_REFERENCE_PROTECTION@ 00000001800054a0     libgetlocal003.obj
 0002:000004c8       ??_C@_0BP@MDKGDGKL@JVMTI_HEAP_REFERENCE_INTERFACE@ 00000001800054c8     libgetlocal003.obj
 0002:000004e8       ??_C@_0CC@JJMIHNJH@JVMTI_HEAP_REFERENCE_STATIC_FIE@ 00000001800054e8     libgetlocal003.obj
 0002:00000510       ??_C@_0CD@IDHEEGID@JVMTI_HEAP_REFERENCE_CONSTANT_P@ 0000000180005510     libgetlocal003.obj
 0002:00000538       ??_C@_0CA@EFFCHNG@JVMTI_HEAP_REFERENCE_SUPERCLASS@ 0000000180005538     libgetlocal003.obj
 0002:00000558       ??_C@_0L@PCDFHGCJ@unknown_11@ 0000000180005558     libgetlocal003.obj
 0002:00000568       ??_C@_0L@NJBICFOK@unknown_12@ 0000000180005568     libgetlocal003.obj
 0002:00000578       ??_C@_0L@MAADBEKL@unknown_13@ 0000000180005578     libgetlocal003.obj
 0002:00000588       ??_C@_0L@IPECICGM@unknown_14@ 0000000180005588     libgetlocal003.obj
 0002:00000598       ??_C@_0L@JGFJLDCN@unknown_15@ 0000000180005598     libgetlocal003.obj
 0002:000005a8       ??_C@_0L@LNHEOAOO@unknown_16@ 00000001800055a8     libgetlocal003.obj
 0002:000005b8       ??_C@_0L@KEGPNBKP@unknown_17@ 00000001800055b8     libgetlocal003.obj
 0002:000005c8       ??_C@_0L@CDPHMNGA@unknown_18@ 00000001800055c8     libgetlocal003.obj
 0002:000005d8       ??_C@_0L@DKOMPMCB@unknown_19@ 00000001800055d8     libgetlocal003.obj
 0002:000005e8       ??_C@_0L@OJGIPJDB@unknown_20@ 00000001800055e8     libgetlocal003.obj
 0002:000005f8       ??_C@_0CA@KAOFNDEM@JVMTI_HEAP_REFERENCE_JNI_GLOBAL@ 00000001800055f8     libgetlocal003.obj
 0002:00000618       ??_C@_0CC@HPFAJBK@JVMTI_HEAP_REFERENCE_SYSTEM_CLA@ 0000000180005618     libgetlocal003.obj
 0002:00000640       ??_C@_0BN@FDEGFOHC@JVMTI_HEAP_REFERENCE_MONITOR@ 0000000180005640     libgetlocal003.obj
 0002:00000660       ??_C@_0CB@HKIBCMAJ@JVMTI_HEAP_REFERENCE_STACK_LOCA@ 0000000180005660     libgetlocal003.obj
 0002:00000688       ??_C@_0BP@EAACMMOE@JVMTI_HEAP_REFERENCE_JNI_LOCAL@ 0000000180005688     libgetlocal003.obj
 0002:000006a8       ??_C@_0BM@IJDEOGOE@JVMTI_HEAP_REFERENCE_THREAD@ 00000001800056a8     libgetlocal003.obj
 0002:000006c8       ??_C@_0BL@EDGPPKC@JVMTI_HEAP_REFERENCE_OTHER@ 00000001800056c8     libgetlocal003.obj
 0002:000006e4       ??_C@_04BCJPDBDA@Code@     00000001800056e4     libgetlocal003.obj
 0002:000006f0       ??_C@_0BA@OCLMCFKC@LineNumberTable@ 00000001800056f0     libgetlocal003.obj
 0002:00000700       ??_C@_0BD@CPAEPILC@LocalVariableTable@ 0000000180005700     libgetlocal003.obj
 0002:00000718       ??_C@_0BH@NMBDNHBD@LocalVariableTypeTable@ 0000000180005718     libgetlocal003.obj
 0002:00000730       ??_C@_0O@HIHEEDNJ@StackMapTable@ 0000000180005730     libgetlocal003.obj
 0002:00000740       ??_C@_0L@HCDIAMJG@?9?5?$CFs?0?5?$CFd?3?5@ 0000000180005740     libgetlocal003.obj
 0002:00000750       ??_C@_0JI@HLPECLFI@?$CD?5?4?4?4?6?$CD?5ERROR?3?5too?5many?5complai@ 0000000180005750     libgetlocal003.obj
 0002:000007f0       ??_C@_0ED@JNEKCCOB@The?5following?5fake?5exception?5st@ 00000001800057f0     libgetlocal003.obj
 0002:00000838       ??_C@_0CN@FCNMDFBH@nsk?4share?4Fake_Exception_for_RU@ 0000000180005838     libgetlocal003.obj
 0002:00000868       ??_C@_08PGFFNAEI@?$CI?$CFs?3?$CFd?$CJ?5@ 0000000180005868     libgetlocal003.obj
 0002:00000878       ??_C@_0DP@IENMAEGI@s?2test?2hotspot?2jtreg?2vmTestbase@ 0000000180005878     libgetlocal003.obj
 0002:000008b8       ??_C@_0BL@NDJLFFJB@?7at?5nsk_lvcomplain?$CI?$CFs?3?$CFd?$CJ?6@ 00000001800058b8     libgetlocal003.obj
 0002:000008d8       ??_C@_0BC@JOOKAFKF@?$CD?5ERROR?3?5?$CFs?0?5?$CFd?3?5@ 00000001800058d8     libgetlocal003.obj
 0002:000008f0       ??_C@_09KJEAHMEH@?$CD?5ERROR?3?5@ 00000001800058f0     libgetlocal003.obj
 0002:000008fc       ??_C@_02GPIOPFAK@?$DO?$DO@ 00000001800058fc     libgetlocal003.obj
 0002:00000900       ??_C@_02FODMEDOG@?$DM?$DM@ 0000000180005900     libgetlocal003.obj
 0002:00000904       ??_C@_02DJGKEECL@?4?4@     0000000180005904     libgetlocal003.obj
 0002:00000908       ??_C@_0O@CJPGJOAF@?9?5?$CFs?0?5?$CFd?3?5?$CFs?5@ 0000000180005908     libgetlocal003.obj
 0002:00000918       ??_C@_0CB@IAKPDOIC@?$CD?5?5?5verified?5assertion?5is?5FALSE@ 0000000180005918     libgetlocal003.obj
 0002:00000940       ??_C@_0CO@LGONDEPD@stdout?3?5fflush?5failed?5?9?5err?$DN?$CFd?5@ 0000000180005940     libgetlocal003.obj
 0002:00000970       ??_C@_0CO@KBGKJPBD@stderr?3?5fflush?5failed?5?9?5err?$DN?$CFd?5@ 0000000180005970     libgetlocal003.obj
 0002:000009a0       ??_C@_0BB@JCNMKLLK@JVMTI_ERROR_NONE@ 00000001800059a0     libgetlocal003.obj
 0002:000009b8       ??_C@_0BL@LDIMKLPH@JVMTI_ERROR_INVALID_THREAD@ 00000001800059b8     libgetlocal003.obj
 0002:000009d8       ??_C@_0CB@PJFPAIKJ@JVMTI_ERROR_INVALID_THREAD_GROU@ 00000001800059d8     libgetlocal003.obj
 0002:00000a00       ??_C@_0BN@LLMKHMNF@JVMTI_ERROR_INVALID_PRIORITY@ 0000000180005a00     libgetlocal003.obj
 0002:00000a20       ??_C@_0CB@MBOFKAGB@JVMTI_ERROR_THREAD_NOT_SUSPENDE@ 0000000180005a20     libgetlocal003.obj
 0002:00000a48       ??_C@_0BN@FABOLPBI@JVMTI_ERROR_THREAD_SUSPENDED@ 0000000180005a48     libgetlocal003.obj
 0002:00000a68       ??_C@_0BN@FDGNOBJM@JVMTI_ERROR_THREAD_NOT_ALIVE@ 0000000180005a68     libgetlocal003.obj
 0002:00000a88       ??_C@_0BL@GOBIFKNJ@JVMTI_ERROR_INVALID_OBJECT@ 0000000180005a88     libgetlocal003.obj
 0002:00000aa8       ??_C@_0BK@FCMAJPPC@JVMTI_ERROR_INVALID_CLASS@ 0000000180005aa8     libgetlocal003.obj
 0002:00000ac8       ??_C@_0BP@IKLLBKEB@JVMTI_ERROR_CLASS_NOT_PREPARED@ 0000000180005ac8     libgetlocal003.obj
 0002:00000ae8       ??_C@_0BN@KLPPLKG@JVMTI_ERROR_INVALID_METHODID@ 0000000180005ae8     libgetlocal003.obj
 0002:00000b08       ??_C@_0BN@BCEKOKND@JVMTI_ERROR_INVALID_LOCATION@ 0000000180005b08     libgetlocal003.obj
 0002:00000b28       ??_C@_0BM@DFDGPME@JVMTI_ERROR_INVALID_FIELDID@ 0000000180005b28     libgetlocal003.obj
 0002:00000b48       ??_C@_0BL@NELIEPEC@JVMTI_ERROR_NO_MORE_FRAMES@ 0000000180005b48     libgetlocal003.obj
 0002:00000b68       ??_C@_0BJ@BDBECFDM@JVMTI_ERROR_OPAQUE_FRAME@ 0000000180005b68     libgetlocal003.obj
 0002:00000b88       ??_C@_0BK@MIIFNLOB@JVMTI_ERROR_TYPE_MISMATCH@ 0000000180005b88     libgetlocal003.obj
 0002:00000ba8       ??_C@_0BJ@HPCAOILC@JVMTI_ERROR_INVALID_SLOT@ 0000000180005ba8     libgetlocal003.obj
 0002:00000bc8       ??_C@_0BG@CHILOPNI@JVMTI_ERROR_DUPLICATE@ 0000000180005bc8     libgetlocal003.obj
 0002:00000be0       ??_C@_0BG@DIEMLHKM@JVMTI_ERROR_NOT_FOUND@ 0000000180005be0     libgetlocal003.obj
 0002:00000bf8       ??_C@_0BM@NHMCKHOB@JVMTI_ERROR_INVALID_MONITOR@ 0000000180005bf8     libgetlocal003.obj
 0002:00000c18       ??_C@_0BO@PPEDAJGL@JVMTI_ERROR_NOT_MONITOR_OWNER@ 0000000180005c18     libgetlocal003.obj
 0002:00000c38       ??_C@_0BG@FCAIPEID@JVMTI_ERROR_INTERRUPT@ 0000000180005c38     libgetlocal003.obj
 0002:00000c50       ??_C@_0CB@EGDBNKOI@JVMTI_ERROR_INVALID_CLASS_FORMA@ 0000000180005c50     libgetlocal003.obj
 0002:00000c78       ??_C@_0CG@DGKOGIAL@JVMTI_ERROR_CIRCULAR_CLASS_DEFI@ 0000000180005c78     libgetlocal003.obj
 0002:00000ca0       ??_C@_0BP@ICEALPKC@JVMTI_ERROR_FAILS_VERIFICATION@ 0000000180005ca0     libgetlocal003.obj
 0002:00000cc0       ??_C@_0DC@JDACLMIO@JVMTI_ERROR_UNSUPPORTED_REDEFIN@ 0000000180005cc0     libgetlocal003.obj
 0002:00000cf8       ??_C@_0DE@GKDKNOMJ@JVMTI_ERROR_UNSUPPORTED_REDEFIN@ 0000000180005cf8     libgetlocal003.obj
 0002:00000d30       ??_C@_0BO@LAFKIOG@JVMTI_ERROR_INVALID_TYPESTATE@ 0000000180005d30     libgetlocal003.obj
 0002:00000d50       ??_C@_0DH@INDGCLLB@JVMTI_ERROR_UNSUPPORTED_REDEFIN@ 0000000180005d50     libgetlocal003.obj
 0002:00000d88       ??_C@_0DE@NHEOMMGI@JVMTI_ERROR_UNSUPPORTED_REDEFIN@ 0000000180005d88     libgetlocal003.obj
 0002:00000dc0       ??_C@_0CA@EKPNJOEP@JVMTI_ERROR_UNSUPPORTED_VERSION@ 0000000180005dc0     libgetlocal003.obj
 0002:00000de0       ??_C@_0BN@OFFMAHHL@JVMTI_ERROR_NAMES_DONT_MATCH@ 0000000180005de0     libgetlocal003.obj
 0002:00000e00       ??_C@_0DN@HHBBLAKE@JVMTI_ERROR_UNSUPPORTED_REDEFIN@ 0000000180005e00     libgetlocal003.obj
 0002:00000e40       ??_C@_0DO@HMBGBGNA@JVMTI_ERROR_UNSUPPORTED_REDEFIN@ 0000000180005e40     libgetlocal003.obj
 0002:00000e80       ??_C@_0BP@PBECGKHJ@JVMTI_ERROR_UNMODIFIABLE_CLASS@ 0000000180005e80     libgetlocal003.obj
 0002:00000ea0       ??_C@_0BK@CANILEHF@JVMTI_ERROR_NOT_AVAILABLE@ 0000000180005ea0     libgetlocal003.obj
 0002:00000ec0       ??_C@_0CE@INJKMEFK@JVMTI_ERROR_MUST_POSSESS_CAPABI@ 0000000180005ec0     libgetlocal003.obj
 0002:00000ee8       ??_C@_0BJ@LBFPFPDM@JVMTI_ERROR_NULL_POINTER@ 0000000180005ee8     libgetlocal003.obj
 0002:00000f08       ??_C@_0BP@CHJPNNEM@JVMTI_ERROR_ABSENT_INFORMATION@ 0000000180005f08     libgetlocal003.obj
 0002:00000f28       ??_C@_0BP@OMFMNLC@JVMTI_ERROR_INVALID_EVENT_TYPE@ 0000000180005f28     libgetlocal003.obj
 0002:00000f48       ??_C@_0BN@BIBNPHHO@JVMTI_ERROR_ILLEGAL_ARGUMENT@ 0000000180005f48     libgetlocal003.obj
 0002:00000f68       ??_C@_0BK@KKNDHDCE@JVMTI_ERROR_NATIVE_METHOD@ 0000000180005f68     libgetlocal003.obj
 0002:00000f88       ??_C@_0BK@PMKCFHAE@JVMTI_ERROR_OUT_OF_MEMORY@ 0000000180005f88     libgetlocal003.obj
 0002:00000fa8       ??_C@_0BK@NNJBDMNB@JVMTI_ERROR_ACCESS_DENIED@ 0000000180005fa8     libgetlocal003.obj
 0002:00000fc8       ??_C@_0BI@GHECLMNC@JVMTI_ERROR_WRONG_PHASE@ 0000000180005fc8     libgetlocal003.obj
 0002:00000fe0       ??_C@_0BF@OLIHJOII@JVMTI_ERROR_INTERNAL@ 0000000180005fe0     libgetlocal003.obj
 0002:00000ff8       ??_C@_0BO@EOHGKJHI@JVMTI_ERROR_UNATTACHED_THREAD@ 0000000180005ff8     libgetlocal003.obj
 0002:00001018       ??_C@_0CA@LKHFDACL@JVMTI_ERROR_INVALID_ENVIRONMENT@ 0000000180006018     libgetlocal003.obj
 0002:00001038       ??_C@_0BA@MMFHLOKK@?$DMunknown?5error?$DO@ 0000000180006038     libgetlocal003.obj
 0002:00001048       ??_C@_0CF@CBHOKDB@throwable?5?$DN?5jni?9?$DOExceptionOccur@ 0000000180006048     libgetlocal003.obj
 0002:00001070       ??_C@_03OFAPEBGM@?$CFs?6@  0000000180006070     libgetlocal003.obj
 0002:00001078       ??_C@_0DM@LPIGEGNJ@s?2test?2hotspot?2jtreg?2vmTestbase@ 0000000180006078     libgetlocal003.obj
 0002:000010b8       ??_C@_0CC@NFCNPEPK@Exception?5in?5JNI?5call?5?$CIcleared?$CJ@ 00000001800060b8     libgetlocal003.obj
 0002:000010e0       ??_C@_0BJ@IBAKFIKF@jni?9?$DOExceptionDescribe?$CI?$CJ@ 00000001800060e0     libgetlocal003.obj
 0002:00001100       ??_C@_0BG@GGKALKMH@jni?9?$DOExceptionClear?$CI?$CJ@ 0000000180006100     libgetlocal003.obj
 0002:00001118       ??_C@_0CF@JMGFGJLJ@?$CD?5?5?5verified?5JNI?5assertion?5is?5F@ 0000000180006118     libgetlocal003.obj
 0002:00001140       ??_C@_0CB@MLNJNCLJ@?5?5jvmti?5error?3?5code?$DN?$CFd?0?5name?$DN?$CFs@ 0000000180006140     libgetlocal003.obj
 0002:00001168       ??_C@_0CD@OHBGDKMK@?$CD?5?5?5jvmti?5error?3?5code?$DN?$CFd?0?5name?$DN@ 0000000180006168     libgetlocal003.obj
 0002:00001190       ??_C@_0CG@JNNCGPHB@?$CD?5?5?5error?5expected?3?5code?$DN?$CFd?0?5na@ 0000000180006190     libgetlocal003.obj
 0002:000011c0       ??_C@_0EB@IMGKPCGE@?$CIstr_obj?5?$DN?5jni?9?$DONewStringUTF?$CIco@ 00000001800061c0     libgetlocal003.obj
 0002:00001210       ??_C@_0EA@HFOGGBCC@s?2test?2hotspot?2jtreg?2vmTestbase@ 0000000180006210     libgetlocal003.obj
 0002:00001250       ??_C@_05KKCIMGE@error@     0000000180006250     libgetlocal003.obj
 0002:00001258       ??_C@_0CJ@JACLEAA@Test?5failed?5by?5setFailStatus?$CI?$CJ?4@ 0000000180006258     libgetlocal003.obj
 0002:00001290       ??_C@_0EA@PNBCDMOA@s?2test?2hotspot?2jtreg?2vmTestbase@ 0000000180006290     libgetlocal003.obj
 0002:000012d0       ??_C@_0DI@ILAHDLMP@?$CI?$CKagentThreadProc?$CJ?$CIjvmti_env?0?5a@ 00000001800062d0     libgetlocal003.obj
 0002:00001308       ??_C@_0BD@KDBALNLB@JVMTI?5agent?5thread@ 0000000180006308     libgetlocal003.obj
 0002:00001320       ??_C@_0BB@NOKBFPFO@java?1lang?1Thread@ 0000000180006320     libgetlocal003.obj
 0002:00001334       ??_C@_06FALKBLGB@?$DMinit?$DO@ 0000000180006334     libgetlocal003.obj
 0002:00001340       ??_C@_0BG@IKDDPPGD@?$CILjava?1lang?1String?$DL?$CJV@ 0000000180006340     libgetlocal003.obj
 0002:00001360       ??_C@_0EB@IFJBFEKC@?$CIthreadClass?5?$DN?5jni_env?9?$DOFindCla@ 0000000180006360     libgetlocal003.obj
 0002:000013b0       ??_C@_0GF@FGFIBKKL@?$CIthreadCtor?5?$DN?5jni_env?9?$DOGetMetho@ 00000001800063b0     libgetlocal003.obj
 0002:00001418       ??_C@_0DN@NCPDJLOG@?$CIthreadName?5?$DN?5jni_env?9?$DONewStrin@ 0000000180006418     libgetlocal003.obj
 0002:00001460       ??_C@_0FE@PFKODBGC@?$CIthreadObject?5?$DN?5jni_env?9?$DONewObj@ 0000000180006460     libgetlocal003.obj
 0002:000014c0       ??_C@_0ED@HOBAHHJI@?$CIthreadGlobalRef?5?$DN?5jni_env?9?$DONew@ 00000001800064c0     libgetlocal003.obj
 0002:00001510       ??_C@_0FN@HNJJAHFC@jvmti_env?9?$DORunAgentThread?$CIagent@ 0000000180006510     libgetlocal003.obj
 0002:00001570       ??_C@_0EA@MOJDNKDF@Debuggee?5status?5sync?5aborted?5be@ 0000000180006570     libgetlocal003.obj
 0002:000015b0       ??_C@_0EA@EEOEJAEN@status?5?$DN?5syncDebuggeeStatus?$CIjni@ 00000001800065b0     libgetlocal003.obj
 0002:000015f0       ??_C@_0BL@JBCFNBMB@nsk_jvmti_resetAgentData?$CI?$CJ@ 00000001800065f0     libgetlocal003.obj
 0002:0000160c       ??_C@_04DIFHPCLD@?$CII?$CJI@ 000000018000660c     libgetlocal003.obj
 0002:00001620       ??_C@_0EL@LPBEELIP@s?2test?2hotspot?2jtreg?2vmTestbase@ 0000000180006620     libgetlocal003.obj
 0002:00001670       ??_C@_0CK@JDAMFDMJ@jvmti?9?$DOSetTag?$CIo?0?5tag?$CJ?5?$DN?$DN?5JVMTI_@ 0000000180006670     libgetlocal003.obj
 0002:000016a0       ??_C@_0CC@DAMNHKNI@Can?8t?5set?5tag?5?$CFli?5for?5object?5?$CFl@ 00000001800066a0     libgetlocal003.obj
 0002:000016c8       ??_C@_0DL@HAJPNKEF@jvmti?9?$DOGetObjectHashCode?$CIo?0?5?$CGha@ 00000001800066c8     libgetlocal003.obj
 0002:00001708       ??_C@_0BL@JFPIEOBF@Can?8t?5get?5hash?5object?5?$CFlx?6@ 0000000180006708     libgetlocal003.obj
 0002:00001728       ??_C@_0BG@DICPHBKN@setTag?3?5?$CF08x?5?$DM?9?5?$CF?53li@ 0000000180006728     libgetlocal003.obj
 0002:00001740       ??_C@_0DH@FCEEBDMJ@?$CIs?5?$DN?5jni?9?$DOGetStringUTFChars?$CIsIn@ 0000000180006740     libgetlocal003.obj
 0002:00001778       ??_C@_0BJ@OKKGHDCN@Can?8t?5get?5string?5at?5?$CF?$CDp?6@ 0000000180006778     libgetlocal003.obj
 0002:00001798       ??_C@_0BP@EKFLGGFJ@Can?8t?5get?5string?5at?5?$CF?$CDp?3?5null?6@ 0000000180006798     libgetlocal003.obj
 0002:000017b8       ??_C@_06ICODBHCL@?5?1?1?5?$CFs@ 00000001800067b8     libgetlocal003.obj
 0002:000017c0       ??_C@_0DB@KGFPLEGO@?$CIr?5?$DN?5jvmti?9?$DOGetTag?$CIo?0?5?$CGtag?$CJ?$CJ?5?$DN?$DN@ 00000001800067c0     libgetlocal003.obj
 0002:000017f8       ??_C@_0CO@PDAGBCGJ@Can?8t?5GetTag?5for?5object?5?$CFlx?4?5Re@ 00000001800067f8     libgetlocal003.obj
 0002:00001828       ??_C@_0CH@HPEODOHC@TEST_BUG?3?5Max?4?5number?5of?5refs?5r@ 0000000180006828     libgetlocal003.obj
 0002:00001850       ??_C@_0DI@PHFCABIM@?$CIr?5?$DN?5jvmti?9?$DOGetTag?$CIfrom?0?5?$CGtagFr@ 0000000180006850     libgetlocal003.obj
 0002:00001888       ??_C@_0DI@MDEGFNKD@TEST_BUG?3?5Can?8t?5GetTag?5for?5obje@ 0000000180006888     libgetlocal003.obj
 0002:000018c0       ??_C@_0DE@MLELJAHM@?$CIr?5?$DN?5jvmti?9?$DOGetTag?$CIto?0?5?$CGtagTo?$CJ?$CJ@ 00000001800068c0     libgetlocal003.obj
 0002:000018f8       ??_C@_0BJ@GENPPCLE@?6?5Var?5name?3?5?$CFs?0?5slot?3?5?$CFd@ 00000001800068f8     libgetlocal003.obj
 0002:00001918       ??_C@_0BD@KKMKIDEF@?0?5start_bci?3?5?$CFI64d@ 0000000180006918     libgetlocal003.obj
 0002:00001930       ??_C@_0BB@MAOHEAJD@?0?5end_bci?3?5?$CFI64d@ 0000000180006930     libgetlocal003.obj
 0002:00001948       ??_C@_0BB@KBHOPJFH@?0?5signature?3?5?$CFs?6@ 0000000180006948     libgetlocal003.obj
 0002:00001960       ??_C@_0BL@FNOFMOJG@?5GetLocalInt?3?5?5?5?5?5?$CFs?5?$CI?$CFd?$CJ?6@ 0000000180006960     libgetlocal003.obj
 0002:00001980       ??_C@_0CO@FPHAGAM@FAIL?3?5GetLocalInt?5failed?5to?5get@ 0000000180006980     libgetlocal003.obj
 0002:000019b0       ??_C@_0EI@JODBMJHB@FAIL?3?5GetLocalInt?5did?5not?5retur@ 00000001800069b0     libgetlocal003.obj
 0002:000019f8       ??_C@_0BL@OKDPJAEJ@?5GetLocalLong?3?5?5?5?5?$CFs?5?$CI?$CFd?$CJ?6@ 00000001800069f8     libgetlocal003.obj
 0002:00001a18       ??_C@_0DA@BPCMDHCL@FAIL?3?5GetLocalLong?5failed?5to?5ge@ 0000000180006a18     libgetlocal003.obj
 0002:00001a50       ??_C@_0GH@KPCMAOMG@FAIL?3?5GetLocalLong?5did?5not?5retu@ 0000000180006a50     libgetlocal003.obj
 0002:00001ab8       ??_C@_0BL@CDMICJKM@?5GetLocalFloat?3?5?5?5?$CFs?5?$CI?$CFd?$CJ?6@ 0000000180006ab8     libgetlocal003.obj
 0002:00001ad8       ??_C@_0DC@DFBIOJEL@FAIL?3?5GetLocalFloat?5failed?5to?5g@ 0000000180006ad8     libgetlocal003.obj
 0002:00001b10       ??_C@_0EM@GCOKADOK@FAIL?3?5GetLocalFloat?5did?5not?5ret@ 0000000180006b10     libgetlocal003.obj
 0002:00001b60       ??_C@_0BL@OLFBDCOD@?5GetLocalDouble?3?5?5?$CFs?5?$CI?$CFd?$CJ?6@ 0000000180006b60     libgetlocal003.obj
 0002:00001b80       ??_C@_0DE@HHJFBAHD@FAIL?3?5GetLocalDouble?5failed?5to?5@ 0000000180006b80     libgetlocal003.obj
 0002:00001bc0       ??_C@_0GL@DGLLBLON@FAIL?3?5GetLocalDouble?5did?5not?5re@ 0000000180006bc0     libgetlocal003.obj
 0002:00001c30       ??_C@_0BL@MIPBHPII@?5GetLocalObject?3?5?5?$CFs?5?$CI?$CFd?$CJ?6@ 0000000180006c30     libgetlocal003.obj
 0002:00001c50       ??_C@_0DE@KHEOPIBH@FAIL?3?5GetLocalObject?5failed?5to?5@ 0000000180006c50     libgetlocal003.obj
 0002:00001c90       ??_C@_0EO@FFENIADE@FAIL?3?5GetLocalObject?5did?5not?5re@ 0000000180006c90     libgetlocal003.obj
 0002:00001ce0       ??_C@_0BE@OPPHNNHO@?7?5failure?3?5?$CFs?5?$CI?$CFd?$CJ?6@ 0000000180006ce0     libgetlocal003.obj
 0002:00001cf8       ??_C@_0DG@OFAAFHAI@?7?5failure?3?5GetFrameLocation?5ret@ 0000000180006cf8     libgetlocal003.obj
 0002:00001d30       ??_C@_0BI@OGEBAPDL@?6?5MethodExit?3?5BEGIN?5?$CFd?6@ 0000000180006d30     libgetlocal003.obj
 0002:00001d48       ??_C@_0BH@NHGFCIAD@?6?5MethodExit?3?5END?5?$CFd?6?6@ 0000000180006d48     libgetlocal003.obj
 0002:00001d60       ??_C@_09OPJEJKBL@printdump@ 0000000180006d60     libgetlocal003.obj
 0002:00001d70       ??_C@_0CJ@KCDEKOCJ@Wrong?5result?5of?5a?5valid?5call?5to@ 0000000180006d70     libgetlocal003.obj
 0002:00001da0       ??_C@_0DG@LAJPGIIE@?$CIGetPotentialCapabilities?$CJ?5unex@ 0000000180006da0     libgetlocal003.obj
 0002:00001dd8       ??_C@_0CN@LKPEOJPO@?$CIAddCapabilities?$CJ?5unexpected?5er@ 0000000180006dd8     libgetlocal003.obj
 0002:00001e08       ??_C@_0CN@BCCBOHCH@?$CIGetCapabilities?$CJ?5unexpected?5er@ 0000000180006e08     libgetlocal003.obj
 0002:00001e38       ??_C@_0DH@HAICLNGL@Warning?3?5Access?5to?5local?5variab@ 0000000180006e38     libgetlocal003.obj
 0002:00001e70       ??_C@_0CO@DJHOJGID@Warning?3?5MethodExit?5event?5is?5no@ 0000000180006e70     libgetlocal003.obj
 0002:00001ea0       ??_C@_0CP@IMINGNLL@?$CISetEventCallbacks?$CJ?5unexpected?5@ 0000000180006ea0     libgetlocal003.obj
 0002:00001ed0       ??_C@_0BM@FFHAFLDP@?6?5Native?5instMeth?3?5started?6@ 0000000180006ed0     libgetlocal003.obj
 0002:00001ef0       ??_C@_0CN@LHLDIOOH@?5Native?5instMeth?3?5GetLocalInsta@ 0000000180006ef0     libgetlocal003.obj
 0002:00001f20       ??_C@_0FA@FHDLKCDB@FAIL?3?5GetLocalInstance?5failed?5t@ 0000000180006f20     libgetlocal003.obj
 0002:00001f70       ??_C@_0FG@DIGFPLJN@FAIL?3?5GetLocalInstance?5returned@ 0000000180006f70     libgetlocal003.obj
 0002:00001fd0       ??_C@_0EO@DMMFABFJ@FAIL?3?5GetLocalInstance?5failed?5t@ 0000000180006fd0     libgetlocal003.obj
 0002:00002020       ??_C@_0FE@BMOJPLFL@FAIL?3?5GetLocalInstance?5returned@ 0000000180007020     libgetlocal003.obj
 0002:00002078       ??_C@_0BN@HEMBLNED@?5Native?5instMeth?3?5finished?6?6@ 0000000180007078     libgetlocal003.obj
 0002:00002098       ??_C@_0BL@JMCECDEL@?6?5Native?5getMeth?3?5started?6@ 0000000180007098     libgetlocal003.obj
 0002:000020b8       ??_C@_0CH@CDOJMNAO@JVMTI?5client?5was?5not?5properly?5l@ 00000001800070b8     libgetlocal003.obj
 0002:000020e0       ??_C@_0L@KNBBJLKG@staticMeth@ 00000001800070e0     libgetlocal003.obj
 0002:000020f0       ??_C@_0CG@CFPPLEPH@Cannot?5find?5Method?5ID?5for?5stati@ 00000001800070f0     libgetlocal003.obj
 0002:00002118       ??_C@_0DD@ELHIJBGO@?$CIGetLocalVariableTable?$CJ?5unexpec@ 0000000180007118     libgetlocal003.obj
 0002:00002150       ??_C@_0CM@DDFHGBIE@Failed?5to?5enable?5metod?5exit?5eve@ 0000000180007150     libgetlocal003.obj
 0002:00002180       ??_C@_0CM@KOGMNKLL@?5Native?5getMeth?3?5GetLocalInstan@ 0000000180007180     libgetlocal003.obj
 0002:000021b0       ??_C@_0GB@EGKIDIMD@FAIL?3?5GetLocalInstance?5failed?5t@ 00000001800071b0     libgetlocal003.obj
 0002:00002220       ??_C@_0FP@IBHHFGGG@FAIL?3?5GetLocalInstance?5failed?5t@ 0000000180007220     libgetlocal003.obj
 0002:00002280       ??_C@_0BM@MJFMNHEM@?5Native?5getMeth?3?5finished?6?6@ 0000000180007280     libgetlocal003.obj
 0002:000022a0       ??_C@_0BD@JJKFNBOK@?6?5checkLoc?3?5START?6@ 00000001800072a0     libgetlocal003.obj
 0002:000022b4       ??_C@_06BMHAHPJE@intArg@   00000001800072b4     libgetlocal003.obj
 0002:000022c0       ??_C@_0BH@EECDDHCE@?5GetLocalInt?3?5?$CFs?5?$CI?$CFd?$CJ?6@ 00000001800072c0     libgetlocal003.obj
 0002:000022d8       ??_C@_0CI@LLPDOIHG@?5failure?3?5JVMTI_ERROR_NONE?5is?5e@ 00000001800072d8     libgetlocal003.obj
 0002:00002300       ??_C@_02OAHAJOFD@pi@       0000000180007300     libgetlocal003.obj
 0002:00002308       ??_C@_0DB@IFGJPPKC@?5failure?3?5JVMTI_ERROR_TYPE_MISM@ 0000000180007308     libgetlocal003.obj
 0002:00002340       ??_C@_0DA@DNPPKBNA@?5failure?3?5JVMTI_ERROR_INVALID_S@ 0000000180007340     libgetlocal003.obj
 0002:00002370       ??_C@_0DK@OMNHPOB@?5failure?3?5locations?5of?5vars?5wit@ 0000000180007370     libgetlocal003.obj
 0002:000023b0       ??_C@_0DO@LADJKMLD@?6?5Success?3?5locations?5of?5vars?5wi@ 00000001800073b0     libgetlocal003.obj
 0002:000023f0       ??_C@_0BC@MCMDCIFI@?6?5checkLoc?3?5END?6?6@ 00000001800073f0     libgetlocal003.obj
 0002:00002420       ??_C@_1EC@JIJBPKFM@?$AAa?$AAp?$AAi?$AA?9?$AAm?$AAs?$AA?9?$AAw?$AAi?$AAn?$AA?9?$AAc?$AAo?$AAr?$AAe@ 0000000180007420     MSVCRT:thread_safe_statics.obj
 0002:00002468       ??_C@_1BK@MGMFAEKH@?$AAk?$AAe?$AAr?$AAn?$AAe?$AAl?$AA3?$AA2?$AA?4?$AAd?$AAl?$AAl@ 0000000180007468     MSVCRT:thread_safe_statics.obj
 0002:00002488       ??_C@_0BJ@JEBJOJFJ@SleepConditionVariableCS@ 0000000180007488     MSVCRT:thread_safe_statics.obj
 0002:000024a8       ??_C@_0BJ@PGPPEPCC@WakeAllConditionVariable@ 00000001800074a8     MSVCRT:thread_safe_statics.obj
 0002:000024c8       _pDefaultRawDllMain        00000001800074c8     MSVCRT:dll_dllmain.obj
 0002:000024c8       _pRawDllMain               00000001800074c8     MSVCRT:dll_dllmain.obj
 0002:000024d0       __xmm@ffffffffffffffffffffffffffffffff 00000001800074d0     MSVCRT:utility.obj
 0002:000024e0       _load_config_used          00000001800074e0     MSVCRT:loadcfg.obj
 0002:00002700       _tls_used                  0000000180007700     MSVCRT:tlssup.obj
 0002:00002728       __volatile_metadata        0000000180007728     <linker-defined>
 0002:00002ae8       __rtc_iaa                  0000000180007ae8     MSVCRT:initsect.obj
 0002:00002af0       __rtc_izz                  0000000180007af0     MSVCRT:initsect.obj
 0002:00002af8       __rtc_taa                  0000000180007af8     MSVCRT:initsect.obj
 0002:00002b00       __rtc_tzz                  0000000180007b00     MSVCRT:initsect.obj
 0002:00002b08       _tls_start                 0000000180007b08     MSVCRT:tlssup.obj
 0002:00002b0c       _Init_thread_epoch         0000000180007b0c     MSVCRT:thread_safe_statics.obj
 0002:00002b10       _tls_end                   0000000180007b10     MSVCRT:tlssup.obj
 0002:000032b0       __IMPORT_DESCRIPTOR_KERNEL32 00000001800082b0     kernel32:KERNEL32.dll
 0002:000032c4       __IMPORT_DESCRIPTOR_VCRUNTIME140 00000001800082c4     vcruntime:VCRUNTIME140.dll
 0002:000032d8       __IMPORT_DESCRIPTOR_api-ms-win-crt-runtime-l1-1-0 00000001800082d8     ucrt:api-ms-win-crt-runtime-l1-1-0.dll
 0002:000032ec       __IMPORT_DESCRIPTOR_api-ms-win-crt-stdio-l1-1-0 00000001800082ec     ucrt:api-ms-win-crt-stdio-l1-1-0.dll
 0002:00003300       __IMPORT_DESCRIPTOR_api-ms-win-crt-string-l1-1-0 0000000180008300     ucrt:api-ms-win-crt-string-l1-1-0.dll
 0002:00003314       __NULL_IMPORT_DESCRIPTOR   0000000180008314     kernel32:KERNEL32.dll
 0003:00000034       _Init_global_epoch         0000000180009034     MSVCRT:thread_safe_statics.obj
 0003:00000040       __security_cookie          0000000180009040     MSVCRT:gs_cookie.obj
 0003:00000048       __security_cookie_complement 0000000180009048     MSVCRT:gs_cookie.obj
 0003:00000050       __scrt_native_dllmain_reason 0000000180009050     MSVCRT:utility.obj
 0003:00000058       __isa_available            0000000180009058     MSVCRT:cpu_disp.obj
 0003:0000005c       __isa_enabled              000000018000905c     MSVCRT:cpu_disp.obj
 0003:00000060       __memset_fast_string_threshold 0000000180009060     MSVCRT:cpu_disp.obj
 0003:00000068       __memset_nt_threshold      0000000180009068     MSVCRT:cpu_disp.obj
 0003:00000070       __scrt_ucrt_dll_is_in_use  0000000180009070     MSVCRT:ucrt_stubs.obj
 0003:00000080       g_wrongHeapCallbacks       0000000180009080     libgetlocal003.obj
 0003:00000100       g_szTagInfo                0000000180009100     libgetlocal003.obj
 0003:00002040       g_tagFlags                 000000018000b040     libgetlocal003.obj
 0003:00002428       g_refsToVerifyCnt          000000018000b428     libgetlocal003.obj
 0003:0000242c       g_fakeUserData             000000018000b42c     libgetlocal003.obj
 0003:00002430       g_tagVisitCount            000000018000b430     libgetlocal003.obj
 0003:000033d0       g_refsToVerify             000000018000c3d0     libgetlocal003.obj
 0003:0001aad0       g_userDataError            0000000180023ad0     libgetlocal003.obj
 0003:0001adc0       ?_OptionsStorage@?1??__local_stdio_printf_options@@9@4_KA 0000000180023dc0     libgetlocal003.obj
 0003:0001b398       _tls_index                 0000000180024398     MSVCRT:tlssup.obj
 0003:0001b3a0       __scrt_current_native_startup_state 00000001800243a0     MSVCRT:utility.obj
 0003:0001b3a8       __scrt_native_startup_lock 00000001800243a8     MSVCRT:utility.obj
 0003:0001b3e8       __scrt_debugger_hook_flag  00000001800243e8     MSVCRT:utility_desktop.obj
 0003:0001b3f0       ?__type_info_root_node@@3U__type_info_node@@A 00000001800243f0     MSVCRT:tncleanup.obj
 0003:0001b400       ?_OptionsStorage@?1??__local_stdio_scanf_options@@9@4_KA 0000000180024400     MSVCRT:default_local_stdio_options.obj
 0003:0001b408       __favor                    0000000180024408     MSVCRT:cpu_disp.obj
 0003:0001b410       __dyn_tls_init_callback    0000000180024410     <common>

 entry point at        0001:00002c20

 Static symbols

 0000:fffd9000       .debug$S                   0000000180000000     getlocal003.exp
 0000:fffd9000       .debug$S                   0000000180000000     vcruntime:VCRUNTIME140.dll
 0000:fffd9000       .debug$S                   0000000180000000     vcruntime:VCRUNTIME140.dll
 0000:fffd9000       .debug$S                   0000000180000000     vcruntime:VCRUNTIME140.dll
 0000:fffd9000       .debug$S                   0000000180000000     vcruntime:VCRUNTIME140.dll
 0000:fffd9000       .debug$S                   0000000180000000     vcruntime:VCRUNTIME140.dll
 0000:fffd9000       .debug$S                   0000000180000000     vcruntime:VCRUNTIME140.dll
 0000:fffd9000       .debug$S                   0000000180000000     vcruntime:VCRUNTIME140.dll
 0000:fffd9000       .debug$S                   0000000180000000     ucrt:api-ms-win-crt-convert-l1-1-0.dll
 0002:ffffb000       .idata$6                   0000000180000000     ucrt:api-ms-win-crt-convert-l1-1-0.dll
 0000:fffd9000       .debug$S                   0000000180000000     ucrt:api-ms-win-crt-heap-l1-1-0.dll
 0000:fffd9000       .debug$S                   0000000180000000     ucrt:api-ms-win-crt-heap-l1-1-0.dll
 0000:fffd9000       .debug$S                   0000000180000000     ucrt:api-ms-win-crt-heap-l1-1-0.dll
 0000:fffd9000       .debug$S                   0000000180000000     ucrt:api-ms-win-crt-heap-l1-1-0.dll
 0002:ffffb000       .idata$6                   0000000180000000     ucrt:api-ms-win-crt-heap-l1-1-0.dll
 0000:fffd9000       .debug$S                   0000000180000000     ucrt:api-ms-win-crt-runtime-l1-1-0.dll
 0000:fffd9000       .debug$S                   0000000180000000     ucrt:api-ms-win-crt-runtime-l1-1-0.dll
 0000:fffd9000       .debug$S                   0000000180000000     ucrt:api-ms-win-crt-runtime-l1-1-0.dll
 0000:fffd9000       .debug$S                   0000000180000000     ucrt:api-ms-win-crt-runtime-l1-1-0.dll
 0000:fffd9000       .debug$S                   0000000180000000     ucrt:api-ms-win-crt-runtime-l1-1-0.dll
 0000:fffd9000       .debug$S                   0000000180000000     ucrt:api-ms-win-crt-runtime-l1-1-0.dll
 0000:fffd9000       .debug$S                   0000000180000000     ucrt:api-ms-win-crt-runtime-l1-1-0.dll
 0000:fffd9000       .debug$S                   0000000180000000     ucrt:api-ms-win-crt-runtime-l1-1-0.dll
 0000:fffd9000       .debug$S                   0000000180000000     ucrt:api-ms-win-crt-runtime-l1-1-0.dll
 0000:fffd9000       .debug$S                   0000000180000000     ucrt:api-ms-win-crt-runtime-l1-1-0.dll
 0000:fffd9000       .debug$S                   0000000180000000     ucrt:api-ms-win-crt-runtime-l1-1-0.dll
 0000:fffd9000       .debug$S                   0000000180000000     ucrt:api-ms-win-crt-runtime-l1-1-0.dll
 0000:fffd9000       .debug$S                   0000000180000000     ucrt:api-ms-win-crt-runtime-l1-1-0.dll
 0000:fffd9000       .debug$S                   0000000180000000     ucrt:api-ms-win-crt-runtime-l1-1-0.dll
 0000:fffd9000       .debug$S                   0000000180000000     ucrt:api-ms-win-crt-runtime-l1-1-0.dll
 0000:fffd9000       .debug$S                   0000000180000000     ucrt:api-ms-win-crt-runtime-l1-1-0.dll
 0000:fffd9000       .debug$S                   0000000180000000     ucrt:api-ms-win-crt-stdio-l1-1-0.dll
 0000:fffd9000       .debug$S                   0000000180000000     ucrt:api-ms-win-crt-stdio-l1-1-0.dll
 0000:fffd9000       .debug$S                   0000000180000000     ucrt:api-ms-win-crt-stdio-l1-1-0.dll
 0000:fffd9000       .debug$S                   0000000180000000     ucrt:api-ms-win-crt-stdio-l1-1-0.dll
 0000:fffd9000       .debug$S                   0000000180000000     ucrt:api-ms-win-crt-stdio-l1-1-0.dll
 0000:fffd9000       .debug$S                   0000000180000000     ucrt:api-ms-win-crt-stdio-l1-1-0.dll
 0000:fffd9000       .debug$S                   0000000180000000     ucrt:api-ms-win-crt-stdio-l1-1-0.dll
 0000:fffd9000       .debug$S                   0000000180000000     ucrt:api-ms-win-crt-stdio-l1-1-0.dll
 0000:fffd9000       .debug$S                   0000000180000000     ucrt:api-ms-win-crt-stdio-l1-1-0.dll
 0000:fffd9000       .debug$S                   0000000180000000     ucrt:api-ms-win-crt-stdio-l1-1-0.dll
 0000:fffd9000       .debug$S                   0000000180000000     ucrt:api-ms-win-crt-string-l1-1-0.dll
 0000:fffd9000       .debug$S                   0000000180000000     ucrt:api-ms-win-crt-string-l1-1-0.dll
 0000:fffd9000       .debug$S                   0000000180000000     ucrt:api-ms-win-crt-string-l1-1-0.dll
 0000:fffd9000       .debug$S                   0000000180000000     ucrt:api-ms-win-crt-string-l1-1-0.dll
 0000:fffd9000       .debug$S                   0000000180000000     ucrt:api-ms-win-crt-string-l1-1-0.dll
 0000:fffd9000       .debug$S                   0000000180000000     ucrt:api-ms-win-crt-string-l1-1-0.dll
 0000:fffd9000       .debug$S                   0000000180000000     ucrt:api-ms-win-crt-string-l1-1-0.dll
 0000:fffd9000       .debug$S                   0000000180000000     ucrt:api-ms-win-crt-string-l1-1-0.dll
 0000:fffd9000       .debug$S                   0000000180000000     kernel32:KERNEL32.dll
 0000:fffd9000       .debug$S                   0000000180000000     kernel32:KERNEL32.dll
 0000:fffd9000       .debug$S                   0000000180000000     kernel32:KERNEL32.dll
 0000:fffd9000       .debug$S                   0000000180000000     kernel32:KERNEL32.dll
 0000:fffd9000       .debug$S                   0000000180000000     kernel32:KERNEL32.dll
 0000:fffd9000       .debug$S                   0000000180000000     kernel32:KERNEL32.dll
 0000:fffd9000       .debug$S                   0000000180000000     kernel32:KERNEL32.dll
 0000:fffd9000       .debug$S                   0000000180000000     kernel32:KERNEL32.dll
 0000:fffd9000       .debug$S                   0000000180000000     kernel32:KERNEL32.dll
 0000:fffd9000       .debug$S                   0000000180000000     kernel32:KERNEL32.dll
 0000:fffd9000       .debug$S                   0000000180000000     kernel32:KERNEL32.dll
 0000:fffd9000       .debug$S                   0000000180000000     kernel32:KERNEL32.dll
 0000:fffd9000       .debug$S                   0000000180000000     kernel32:KERNEL32.dll
 0000:fffd9000       .debug$S                   0000000180000000     kernel32:KERNEL32.dll
 0000:fffd9000       .debug$S                   0000000180000000     kernel32:KERNEL32.dll
 0000:fffd9000       .debug$S                   0000000180000000     kernel32:KERNEL32.dll
 0000:fffd9000       .debug$S                   0000000180000000     kernel32:KERNEL32.dll
 0000:fffd9000       .debug$S                   0000000180000000     kernel32:KERNEL32.dll
 0000:fffd9000       .debug$S                   0000000180000000     kernel32:KERNEL32.dll
 0000:fffd9000       .debug$S                   0000000180000000     kernel32:KERNEL32.dll
 0000:fffd9000       .debug$S                   0000000180000000     kernel32:KERNEL32.dll
 0000:fffd9000       .debug$S                   0000000180000000     kernel32:KERNEL32.dll
 0000:fffd9000       .debug$S                   0000000180000000     kernel32:KERNEL32.dll
 0000:fffd9000       .debug$S                   0000000180000000     kernel32:KERNEL32.dll
 0000:fffd9000       .debug$S                   0000000180000000     kernel32:KERNEL32.dll
 0000:fffd9000       .debug$S                   0000000180000000     kernel32:KERNEL32.dll
 0000:fffd9000       .debug$S                   0000000180000000     kernel32:KERNEL32.dll
 0000:fffd9000       .debug$S                   0000000180000000     kernel32:KERNEL32.dll
 0001:000013e8       MethodExit                 00000001800023e8 f   libgetlocal003.obj
 0001:000014e4       addRefToVerify             00000001800024e4 f   libgetlocal003.obj
 0001:00001550       agentThreadWrapper         0000000180002550 f   libgetlocal003.obj
 0001:00001740       file_basename              0000000180002740 f   libgetlocal003.obj
 0001:00001e00       startAgentThreadWrapper    0000000180002e00 f   libgetlocal003.obj
 0001:00002140       syncDebuggeeStatus         0000000180003140 f   libgetlocal003.obj
 0001:000022d8       test_locals                00000001800032d8 f   libgetlocal003.obj
 0001:000026dc       capture_previous_context   00000001800036dc f   MSVCRT:gs_report.obj
 0001:00002750       ?__scrt_initialize_thread_safe_statics@@YAHXZ 0000000180003750 f   MSVCRT:thread_safe_statics.obj
 0001:00002820       ?__scrt_uninitialize_thread_safe_statics@@YAXXZ 0000000180003820 f   MSVCRT:thread_safe_statics.obj
 0001:000028d0       $$000000                   00000001800038d0     MSVCRT:amdsecgs.obj
 0001:00002900       ?dllmain_crt_dispatch@@YAHQEAUHINSTANCE__@@KQEAX@Z 0000000180003900 f   MSVCRT:dll_dllmain.obj
 0001:00002950       ?dllmain_crt_process_attach@@YAHQEAUHINSTANCE__@@QEAX@Z 0000000180003950 f   MSVCRT:dll_dllmain.obj
 0001:00002a68       ?dllmain_crt_process_detach@@YAH_N@Z 0000000180003a68 f   MSVCRT:dll_dllmain.obj
 0001:00002aec       ?dllmain_dispatch@@YAHQEAUHINSTANCE__@@KQEAX@Z 0000000180003aec f   MSVCRT:dll_dllmain.obj
 0001:00003500       $$000000                   0000000180004500     MSVCRT:guard_dispatch.obj
 0001:00003520       $$000000                   0000000180004520     MSVCRT:guard_xfg_dispatch.obj
 0001:00003536       ?fin$0@?0??dllmain_crt_process_attach@@YAHQEAUHINSTANCE__@@QEAX@Z@4HA 0000000180004536 f   MSVCRT:dll_dllmain.obj
 0001:0000354d       ?fin$0@?0??dllmain_crt_process_detach@@YAH_N@Z@4HA 000000018000454d f   MSVCRT:dll_dllmain.obj
 0001:00003566       ?fin$1@?0??dllmain_crt_process_detach@@YAH_N@Z@4HA 0000000180004566 f   MSVCRT:dll_dllmain.obj
 0001:0000357a       ?filt$0@?0??dllmain_dispatch@@YAHQEAUHINSTANCE__@@KQEAX@Z@4HA 000000018000457a f   MSVCRT:dll_dllmain.obj
 0001:000035b0       __scrt_is_nonwritable_in_current_image$filt$0 00000001800045b0 f   MSVCRT:utility.obj
 0002:000001e8       ?__scrt_initialize_tss_var@@3P6AHXZEA 00000001800051e8     MSVCRT:thread_safe_statics.obj
 0002:00000310       ?opcLengths@@3QBEB         0000000180005310     libgetlocal003.obj
 0002:00002408       GS_ExceptionPointers       0000000180007408     MSVCRT:gs_report.obj
 0002:00002b18       $unwind$fprintf            0000000180007b18     libgetlocal003.obj
 0002:00002b24       $unwind$printf             0000000180007b24     libgetlocal003.obj
 0002:00002b30       $unwind$?NewObject@JNIEnv_@@QEAAPEAV_jobject@@PEAV_jclass@@PEAU_jmethodID@@ZZ 0000000180007b30     libgetlocal003.obj
 0002:00002b30       $unwind$nsk_lcomplain      0000000180007b30     libgetlocal003.obj
 0002:00002b30       $unwind$nsk_ldisplay       0000000180007b30     libgetlocal003.obj
 0002:00002b38       $unwind$Java_nsk_jvmti_unit_GetLocalVariable_getlocal003_getMeth 0000000180007b38     libgetlocal003.obj
 0002:00002b38       $unwind$nsk_lvdisplay      0000000180007b38     libgetlocal003.obj
 0002:00002b38       $unwind$_RTC_Initialize    0000000180007b38     MSVCRT:initsect.obj
 0002:00002b38       $unwind$_RTC_Terminate     0000000180007b38     MSVCRT:initsect.obj
 0002:00002b38       $unwind$?__scrt_initialize_thread_safe_statics@@YAHXZ 0000000180007b38     MSVCRT:thread_safe_statics.obj
 0002:00002b44       $unwind$nsk_lvcomplain     0000000180007b44     libgetlocal003.obj
 0002:00002b5c       $unwind$nsk_ltrace         0000000180007b5c     libgetlocal003.obj
 0002:00002b5c       $unwind$__report_gsfailure 0000000180007b5c     MSVCRT:gs_report.obj
 0002:00002b64       $unwind$Agent_Initialize   0000000180007b64     libgetlocal003.obj
 0002:00002b64       $unwind$nsk_lvtrace        0000000180007b64     libgetlocal003.obj
 0002:00002b64       $unwind$print_LocalVariableEntry 0000000180007b64     libgetlocal003.obj
 0002:00002b64       $unwind$__raise_securityfailure 0000000180007b64     MSVCRT:gs_report.obj
 0002:00002b64       $unwind$__scrt_initialize_crt 0000000180007b64     MSVCRT:utility.obj
 0002:00002b64       $unwind$__scrt_initialize_onexit_tables 0000000180007b64     MSVCRT:utility.obj
 0002:00002b64       $unwind$__scrt_release_startup_lock 0000000180007b64     MSVCRT:utility.obj
 0002:00002b64       $unwind$__scrt_uninitialize_crt 0000000180007b64     MSVCRT:utility.obj
 0002:00002b64       $unwind$_onexit            0000000180007b64     MSVCRT:utility.obj
 0002:00002b6c       $unwind$nsk_lverify        0000000180007b6c     libgetlocal003.obj
 0002:00002b7c       $unwind$nsk_vprintf        0000000180007b7c     libgetlocal003.obj
 0002:00002b8c       $unwind$nsk_printf         0000000180007b8c     libgetlocal003.obj
 0002:00002b94       $unwind$?nsk_jni_lverify@@YAHHPEAUJNIEnv_@@HQEBDH1ZZ 0000000180007b94     libgetlocal003.obj
 0002:00002ba8       $unwind$?nsk_jni_check_exception@@YAHPEAUJNIEnv_@@QEBDH@Z 0000000180007ba8     libgetlocal003.obj
 0002:00002bc4       $unwind$Java_nsk_jvmti_unit_FollowReferences_FollowRefObjects_resetTags 0000000180007bc4     libgetlocal003.obj
 0002:00002bc4       $unwind$addRefToVerify     0000000180007bc4     libgetlocal003.obj
 0002:00002bc4       $unwind$nsk_jvmti_resetAgentData 0000000180007bc4     libgetlocal003.obj
 0002:00002bc4       $unwind$nsk_jvmti_setFailStatus 0000000180007bc4     libgetlocal003.obj
 0002:00002bc4       $unwind$__scrt_initialize_default_local_stdio_options 0000000180007bc4     MSVCRT:default_local_stdio_options.obj
 0002:00002bc4       $unwind$?dllmain_crt_dispatch@@YAHQEAUHINSTANCE__@@KQEAX@Z 0000000180007bc4     MSVCRT:dll_dllmain.obj
 0002:00002bc4       $unwind$DllMain            0000000180007bc4     MSVCRT:dll_dllmain_stub.obj
 0002:00002bc4       $unwind$__GSHandlerCheck   0000000180007bc4     MSVCRT:gshandler.obj
 0002:00002bc4       $unwind$?__scrt_uninitialize_thread_safe_statics@@YAXXZ 0000000180007bc4     MSVCRT:thread_safe_statics.obj
 0002:00002bc4       $unwind$__scrt_acquire_startup_lock 0000000180007bc4     MSVCRT:utility.obj
 0002:00002bc4       $unwind$__scrt_dllmain_after_initialize_c 0000000180007bc4     MSVCRT:utility.obj
 0002:00002bc4       $unwind$__scrt_dllmain_before_initialize_c 0000000180007bc4     MSVCRT:utility.obj
 0002:00002bc4       $unwind$__scrt_dllmain_crt_thread_attach 0000000180007bc4     MSVCRT:utility.obj
 0002:00002bc4       $unwind$__scrt_dllmain_crt_thread_detach 0000000180007bc4     MSVCRT:utility.obj
 0002:00002bc4       $unwind$__scrt_dllmain_uninitialize_c 0000000180007bc4     MSVCRT:utility.obj
 0002:00002bc4       $unwind$__scrt_dllmain_uninitialize_critical 0000000180007bc4     MSVCRT:utility.obj
 0002:00002bc4       $unwind$atexit             0000000180007bc4     MSVCRT:utility.obj
 0002:00002bcc       $unwind$nsk_jvmti_lverify  0000000180007bcc     libgetlocal003.obj
 0002:00002be0       $unwind$exitOnError        0000000180007be0     libgetlocal003.obj
 0002:00002bf0       $unwind$Java_nsk_share_jvmti_ArgumentHandler_getAgentOptionsString 0000000180007bf0     libgetlocal003.obj
 0002:00002c04       $unwind$Java_nsk_jvmti_unit_FollowReferences_FollowRefObjects_getTag 0000000180007c04     libgetlocal003.obj
 0002:00002c04       $unwind$Java_nsk_share_jvmti_DebugeeClass_checkStatus 0000000180007c04     libgetlocal003.obj
 0002:00002c04       $unwind$agentThreadWrapper 0000000180007c04     libgetlocal003.obj
 0002:00002c14       $unwind$startAgentThreadWrapper 0000000180007c14     libgetlocal003.obj
 0002:00002c30       $unwind$syncDebuggeeStatus 0000000180007c30     libgetlocal003.obj
 0002:00002c30       $unwind$__scrt_dllmain_exception_filter 0000000180007c30     MSVCRT:utility.obj
 0002:00002c44       $unwind$Java_nsk_share_jvmti_DebugeeClass_resetAgentData 0000000180007c44     libgetlocal003.obj
 0002:00002c4c       $unwind$MA_checkStatus     0000000180007c4c     libgetlocal003.obj
 0002:00002c60       $unwind$Java_nsk_jvmti_unit_FollowReferences_FollowRefObjects_setTag 0000000180007c60     libgetlocal003.obj
 0002:00002c78       $unwind$Java_nsk_jvmti_unit_FollowReferences_FollowRefObjects_addRefToVerify 0000000180007c78     libgetlocal003.obj
 0002:00002c94       $unwind$test_locals        0000000180007c94     libgetlocal003.obj
 0002:00002cb0       $unwind$MethodExit         0000000180007cb0     libgetlocal003.obj
 0002:00002cc0       $unwind$Java_nsk_jvmti_unit_GetLocalVariable_getlocal003_instMeth 0000000180007cc0     libgetlocal003.obj
 0002:00002cd0       $unwind$Java_nsk_jvmti_unit_GetLocalVariable_getlocal003_checkLoc 0000000180007cd0     libgetlocal003.obj
 0002:00002ce8       $unwind$capture_previous_context 0000000180007ce8     MSVCRT:gs_report.obj
 0002:00002cf4       $unwind$__GSHandlerCheckCommon 0000000180007cf4     MSVCRT:gshandler.obj
 0002:00002d00       $xdatasym                  0000000180007d00     MSVCRT:amdsecgs.obj
 0002:00002d04       $unwind$?dllmain_crt_process_attach@@YAHQEAUHINSTANCE__@@QEAX@Z 0000000180007d04     MSVCRT:dll_dllmain.obj
 0002:00002d40       $unwind$?fin$0@?0??dllmain_crt_process_attach@@YAHQEAUHINSTANCE__@@QEAX@Z@4HA 0000000180007d40     MSVCRT:dll_dllmain.obj
 0002:00002d40       $unwind$?fin$0@?0??dllmain_crt_process_detach@@YAH_N@Z@4HA 0000000180007d40     MSVCRT:dll_dllmain.obj
 0002:00002d40       $unwind$?fin$1@?0??dllmain_crt_process_detach@@YAH_N@Z@4HA 0000000180007d40     MSVCRT:dll_dllmain.obj
 0002:00002d48       $unwind$?dllmain_crt_process_detach@@YAH_N@Z 0000000180007d48     MSVCRT:dll_dllmain.obj
 0002:00002d9c       $unwind$?dllmain_dispatch@@YAHQEAUHINSTANCE__@@KQEAX@Z 0000000180007d9c     MSVCRT:dll_dllmain.obj
 0002:00002dc4       $unwind$?filt$0@?0??dllmain_dispatch@@YAHQEAUHINSTANCE__@@KQEAX@Z@4HA 0000000180007dc4     MSVCRT:dll_dllmain.obj
 0002:00002dcc       $unwind$_DllMainCRTStartup 0000000180007dcc     MSVCRT:dll_dllmain.obj
 0002:00002ddc       $unwind$__scrt_is_nonwritable_in_current_image 0000000180007ddc     MSVCRT:utility.obj
 0002:00002dfc       $unwind$__scrt_is_nonwritable_in_current_image$filt$0 0000000180007dfc     MSVCRT:utility.obj
 0002:00002e04       $unwind$__scrt_fastfail    0000000180007e04     MSVCRT:utility_desktop.obj
 0002:00002e14       $unwind$__security_init_cookie 0000000180007e14     MSVCRT:gs_support.obj
 0002:00002e20       $unwind$__isa_available_init 0000000180007e20     MSVCRT:cpu_disp.obj
 0002:00002e30       $xdatasym                  0000000180007e30     MSVCRT:guard_dispatch.obj
 0002:00002e38       $xdatasym                  0000000180007e38     MSVCRT:guard_xfg_dispatch.obj
 0002:00002e40       .edata                     0000000180007e40     getlocal003.exp
 0002:00002e68       rgpv                       0000000180007e68     getlocal003.exp
 0002:00002eb0       rgszName                   0000000180007eb0     getlocal003.exp
 0002:00002ef8       rgwOrd                     0000000180007ef8     getlocal003.exp
 0002:00002f1c       szName                     0000000180007f1c     getlocal003.exp
 0002:00002f2c       $N00001                    0000000180007f2c     getlocal003.exp
 0002:00002f3b       $N00002                    0000000180007f3b     getlocal003.exp
 0002:00002f48       $N00003                    0000000180007f48     getlocal003.exp
 0002:00002f8d       $N00004                    0000000180007f8d     getlocal003.exp
 0002:00002fca       $N00005                    0000000180007fca     getlocal003.exp
 0002:00003012       $N00006                    0000000180008012     getlocal003.exp
 0002:00003052       $N00007                    0000000180008052     getlocal003.exp
 0002:0000308f       $N00008                    000000018000808f     getlocal003.exp
 0002:000030c9       $N00009                    00000001800080c9     getlocal003.exp
 0002:00003102       $N00010                    0000000180008102     getlocal003.exp
 0002:0000313a       $N00011                    000000018000813a     getlocal003.exp
 0002:00003174       $N00012                    0000000180008174     getlocal003.exp
 0002:000031af       $N00013                    00000001800081af     getlocal003.exp
 0002:000031dd       $N00014                    00000001800081dd     getlocal003.exp
 0002:0000320e       $N00015                    000000018000820e     getlocal003.exp
 0002:0000323d       $N00016                    000000018000823d     getlocal003.exp
 0002:0000326c       $N00017                    000000018000826c     getlocal003.exp
 0002:000032a1       $N00018                    00000001800082a1     getlocal003.exp
 0002:000036aa       .idata$6                   00000001800086aa     kernel32:KERNEL32.dll
 0002:0000370e       .idata$6                   000000018000870e     vcruntime:VCRUNTIME140.dll
 0002:0000387a       .idata$6                   000000018000887a     ucrt:api-ms-win-crt-runtime-l1-1-0.dll
 0002:0000389c       .idata$6                   000000018000889c     ucrt:api-ms-win-crt-stdio-l1-1-0.dll
 0002:000038bc       .idata$6                   00000001800088bc     ucrt:api-ms-win-crt-string-l1-1-0.dll
 0003:00000000       ?codeAttributeName@@3PEBDEB 0000000180009000     libgetlocal003.obj
 0003:00000008       ?lineNumberAttributeName@@3PEBDEB 0000000180009008     libgetlocal003.obj
 0003:00000010       ?localVarAttributeName@@3PEBDEB 0000000180009010     libgetlocal003.obj
 0003:00000018       ?localVarTypeAttributeName@@3PEBDEB 0000000180009018     libgetlocal003.obj
 0003:00000020       ?stackMapAttributeName@@3PEBDEB 0000000180009020     libgetlocal003.obj
 0003:00000028       ?callBytes@@3PAEA          0000000180009028     libgetlocal003.obj
 0003:0000002c       ?allocBytes@@3PAEA         000000018000902c     libgetlocal003.obj
 0003:00000030       methodExitCnt              0000000180009030     libgetlocal003.obj
 0003:0001aad4       redefineAttempted          0000000180023ad4     libgetlocal003.obj
 0003:0001aad8       nsk_context                0000000180023ad8     libgetlocal003.obj
 0003:0001aae4       redefineSucceed            0000000180023ae4     libgetlocal003.obj
 0003:0001aae8       agentFailed                0000000180023ae8     libgetlocal003.obj
 0003:0001aaec       currentAgentStatus         0000000180023aec     libgetlocal003.obj
 0003:0001aaf0       context                    0000000180023af0     libgetlocal003.obj
 0003:0001aba8       agentThread                0000000180023ba8     libgetlocal003.obj
 0003:0001abb0       agentThreadProc            0000000180023bb0     libgetlocal003.obj
 0003:0001abb8       agentThreadArg             0000000180023bb8     libgetlocal003.obj
 0003:0001abc0       agent_data                 0000000180023bc0     libgetlocal003.obj
 0003:0001abd0       jvmti_env                  0000000180023bd0     libgetlocal003.obj
 0003:0001abd8       jvm                        0000000180023bd8     libgetlocal003.obj
 0003:0001abe0       jni_env                    0000000180023be0     libgetlocal003.obj
 0003:0001abe8       checkStatus_func           0000000180023be8     libgetlocal003.obj
 0003:0001abf0       ?codeAttributeIndex@@3GA   0000000180023bf0     libgetlocal003.obj
 0003:0001abf2       printdump                  0000000180023bf2     libgetlocal003.obj
 0003:0001abf4       ?lineNumberAttributeIndex@@3GA 0000000180023bf4     libgetlocal003.obj
 0003:0001abf8       ?localVarAttributeIndex@@3GA 0000000180023bf8     libgetlocal003.obj
 0003:0001abfc       ?localVarTypeAttributeIndex@@3GA 0000000180023bfc     libgetlocal003.obj
 0003:0001ac00       ?stackMapAttributeIndex@@3GA 0000000180023c00     libgetlocal003.obj
 0003:0001ac04       ?stackFrameOffset@@3GA     0000000180023c04     libgetlocal003.obj
 0003:0001ac08       ?mode@@3HA                 0000000180023c08     libgetlocal003.obj
 0003:0001ac0c       ?constantPoolSize@@3GA     0000000180023c0c     libgetlocal003.obj
 0003:0001ac10       ?orig@@3PEBEEB             0000000180023c10     libgetlocal003.obj
 0003:0001ac18       ?gen@@3PEAEEA              0000000180023c18     libgetlocal003.obj
 0003:0001ac20       ?inputPos@@3PEAEEA         0000000180023c20     libgetlocal003.obj
 0003:0001ac28       ?endPos@@3PEBEEB           0000000180023c28     libgetlocal003.obj
 0003:0001ac30       ?genPos@@3PEAEEA           0000000180023c30     libgetlocal003.obj
 0003:0001ac38       ?markPos@@3PEAEEA          0000000180023c38     libgetlocal003.obj
 0003:0001ac40       ?constantPool@@3PEAPEADEA  0000000180023c40     libgetlocal003.obj
 0003:0001ac48       ?constantPoolCount@@3GA    0000000180023c48     libgetlocal003.obj
 0003:0001ac4c       ?zeroBytes@@3PAEA          0000000180023c4c     libgetlocal003.obj
 0003:0001ac50       ?codeLength@@3IA           0000000180023c50     libgetlocal003.obj
 0003:0001ac54       result                     0000000180023c54     libgetlocal003.obj
 0003:0001ac58       ?map@@3PEAIEA              0000000180023c58     libgetlocal003.obj
 0003:0001ac60       ?widening@@3PEACEA         0000000180023c60     libgetlocal003.obj
 0003:0001ac68       jvmti                      0000000180023c68     libgetlocal003.obj
 0003:0001ac70       callbacks                  0000000180023c70     libgetlocal003.obj
 0003:0001ada8       mid                        0000000180023da8     libgetlocal003.obj
 0003:0001adb0       table                      0000000180023db0     libgetlocal003.obj
 0003:0001adb8       entryCount                 0000000180023db8     libgetlocal003.obj
 0003:0001adc8       ?caps@?1??Agent_Initialize@@9@4UjvmtiCapabilities@@A 0000000180023dc8     libgetlocal003.obj
 0003:0001ade0       GS_ExceptionRecord         0000000180023de0     MSVCRT:gs_report.obj
 0003:0001ae80       GS_ContextRecord           0000000180023e80     MSVCRT:gs_report.obj
 0003:0001b350       ?g_tss_cv@@3U_RTL_CONDITION_VARIABLE@@A 0000000180024350     MSVCRT:thread_safe_statics.obj
 0003:0001b358       ?g_tss_event@@3PEAXEA      0000000180024358     MSVCRT:thread_safe_statics.obj
 0003:0001b360       ?g_tss_mutex@@3U_RTL_CRITICAL_SECTION@@A 0000000180024360     MSVCRT:thread_safe_statics.obj
 0003:0001b388       ?g_sleep_condition_variable_cs@@3P6AHPEAU_RTL_CONDITION_VARIABLE@@PEAU_RTL_CRITICAL_SECTION@@K@ZEA 0000000180024388     MSVCRT:thread_safe_statics.obj
 0003:0001b390       ?g_wake_all_condition_variable@@3P6AXPEAU_RTL_CONDITION_VARIABLE@@@ZEA 0000000180024390     MSVCRT:thread_safe_statics.obj
 0003:0001b39c       ?__proc_attached@@3HA      000000018002439c     MSVCRT:dll_dllmain.obj
 0003:0001b3b0       ?is_initialized_as_dll@@3_NA 00000001800243b0     MSVCRT:utility.obj
 0003:0001b3b1       ?module_local_atexit_table_initialized@@3_NA 00000001800243b1     MSVCRT:utility.obj
 0003:0001b3b8       ?module_local_atexit_table@@3U_onexit_table_t@@A 00000001800243b8     MSVCRT:utility.obj
 0003:0001b3d0       ?module_local_at_quick_exit_table@@3U_onexit_table_t@@A 00000001800243d0     MSVCRT:utility.obj
